:020000040800F2
:10000000A0660020290200085B2600087D23000866
:100010005926000859080008094700080000000098
:10002000000000000000000000000000D9270008C8
:10003000350A000800000000D727000855280008EE
:10004000430200084302000843020008430200087C
:100050004302000843020008370A00084302000870
:100060003D0A0008430A0008490A00084302000844
:10007000430200084302000843020008430200084C
:10008000430200084302000843020008430200083C
:10009000430200084302000843020008430200082C
:1000A000430200084302000843020008430200081C
:1000B00043020008FD28000843020008430200082C
:1000C00043020008430200084302000843020008FC
:1000D00043020008430200084302000843020008EC
:1000E00043020008430200084302000843020008DC
:1000F00043020008430200084302000843020008CC
:1001000043020008430200084302000843020008BB
:1001100043020008430200084302000843020008AB
:10012000430200084302000843020008430200089B
:10013000430200084302000843020008430200088B
:10014000430200084302000843020008430200087B
:10015000430200084302000843020008430200086B
:10016000430200084302000843020008430200085B
:10017000430200085D26000843020008000000005A
:10018000430200084302000800F002F800F03CF8C7
:100190000AA090E8000C82448344AAF10107DA45E2
:1001A00001D100F031F8AFF2090EBAE80F0013F0F8
:1001B000010F18BFFB1A43F0010318472046000047
:1001C00040460000103A24BF78C878C1FAD85207D8
:1001D00024BF30C830C144BF04680C6070470000C1
:1001E0000023002400250026103A28BF78C1FBD840
:1001F000520728BF30C148BF0B6070471FB504F0DD
:10020000DBFA1FBD10B510BD00F003F91146FFF772
:10021000F5FF04F0A5FA00F021F903B4FFF7F2FFAF
:1002200003BC04F082FA00000948804709480047EF
:10023000FEE7FEE7FEE7FEE7FEE7FEE7FEE7FEE796
:10024000FEE7FEE704480549054A064B70470000F3
:10025000ED28000889010008A05E0020A0660020AB
:10026000A0620020A0620020704753EA020C00F058
:1002700069802DE9F04B4FF00006002B1FBFB3FA49
:1002800083F503FA05F424FA05F65E4012BF16431F
:10029000B2FA82F502FA05F4C5F120051EBF22FA72
:1002A00005FC44EA0C04203556EA044C4FEA144499
:1002B00018BF641C4FF000084FF00009904271EB2A
:1002C000030C39D3002919BFB1FA81F701FA07F6F7
:1002D000B0FA80F700FA07F6C7F120071EBF20FA30
:1002E00007FC46EA0C062037B6FBF4FCA7EB050733
:1002F000103F07F01F0BCBF120060CFA0BFB2CFA7A
:1003000006F644BFB3460026202FA4BF5E464FF03A
:10031000000B5BEA060C08BF4FF0010B19EB0B0951
:10032000ABFB027C48EB0608C01B06FB02CC0BFBB8
:1003300003CC71EB0C01C1E70B460246414648462F
:10034000BDE8F08B13B54FF000004FF00001AFF3A4
:100350000080BDE81C40704710B5203AC0F00B800B
:10036000B1E81850203AA0E81850B1E81850A0E8B9
:100370001850BFF4F5AF5FEA027C24BFB1E8185013
:10038000A0E8185044BF18C918C0BDE810405FEA83
:10039000827C24BF51F8043B40F8043B08BF7047FF
:1003A000D20728BF31F8023B48BF11F8012B28BF04
:1003B00020F8023B48BF00F8012B70474FF00002C5
:1003C00000B5134694469646203922BFA0E80C504B
:1003D000A0E80C50B1F12001BFF4F7AF090728BF26
:1003E000A0E80C5048BF0CC05DF804EB890028BFA2
:1003F00040F8042B08BF704748BF20F8022B11F0CB
:10040000804F18BF00F8012B704770477047704746
:100410007047754600F02CF8AE4605006946534615
:1004200020F00700854618B020B5FFF70BFFBDE8A8
:1004300020404FF000064FF000074FF000084FF04B
:10044000000B21F00701AC46ACE8C009ACE8C009DC
:10045000ACE8C009ACE8C0098D46704710B5044649
:10046000AFF300802046BDE81040FFF7D6BE000085
:1004700000487047405E002010B5012004F056F996
:1004800000F076F90B4C01220421204600F009FC13
:1004900000226115084800F004FC002208212046D3
:1004A00000F0FFFB002000F07BF9BDE8104000F0F9
:1004B0005FB9000000100240000402402DE9F0473F
:1004C000394E04468021304600F0E6FB05464021C7
:1004D000304600F0E1FB45EA40050421304600F0DB
:1004E000DBFB45EA8006314D4FF40049494628467A
:1004F00000F0D2FB46EAC0062915284600F0CCFBE6
:1005000046EA00176E153146284600F0C5FB47EA5B
:1005100040174FF480784146284600F0BDFB244D3B
:1005200047EA80173146284600F0B6FB47EAC01676
:100530004146284600F0B0FB46EA002680212846C6
:1005400000F0AAFB46EA40264021284600F0A4FB22
:10055000184D46EA80264146284600F09DFB46EAB3
:10056000C0268021284600F097FB46EA003640214D
:10057000284600F091FB104D46EA40364946284691
:1005800000F08AFB46EA80364FF48041284600F0AE
:1005900083FB0A4946EAC0304880000A2070887808
:1005A0006070BDE8F0870000000C024000000240CF
:1005B000000802400018024000040240060100202A
:1005C000F0B53B4887B00024016841F001010160AB
:1005D000016801F001010591016841F0020101602B
:1005E000016801F002010591016841F00401016018
:1005F000016801F004010591016841F00801016002
:10060000016801F008010591016841F010010160E5
:10061000016801F010010591016841F0400101609D
:100620000068022500F040000590C420009001946D
:1006300069462048CDE9024500F036FA4FF40740FC
:10064000009069461C4800F02FFA4FF4707000903B
:1006500069461A4800F028FA4FF43C60184E0090A2
:100660006946304600F020FA4FF44040154F0090A4
:100670006946384600F018FA01A9012081E83100E6
:100680004FF4407000906946384600F00DFA7C2027
:10069000009069460C4800F007FA4FF4E0400090E3
:1006A0006946304600F000FAFFF7E6FE07B0F0BDFD
:1006B00030380240000C02400000024000080240B6
:1006C0000018024000040240001002402DE9F047EB
:1006D0000122254C804615032946204600F0E1FA08
:1006E000012256033146204600F0DBFA00F09EF866
:1006F000E7143946204600F0CFFA0028F9D100224D
:10070000A9462946204600F0CCFA00223146204670
:1007100000F0C7FA154F002505EB0520398801EBDD
:10072000800101EB0800FFF7C9FE01223146204697
:1007300000F0B7FA00223146204600F0B2FA6D1CF4
:10074000082DE9DB38880122801C38804946204684
:1007500000F0A7FA01223146204600F0A2FABDE8D7
:10076000F04700F07DB800000018024006010020AC
:1007700070B50A4D4FF4804400222146284600F00F
:1007800090FA01222146284600F08BFA214628469D
:10079000BDE87040002200F084BA0000001802405A
:1007A00010B5214C08281ED006DC90B1022812D0CA
:1007B000042837D1002206E0102825D020282AD08E
:1007C00040282FD101221021204600F06AFA012290
:1007D00003E0002219E000221EE02021204600F064
:1007E00060FA00220AE000221021204600F059FAA7
:1007F00001222021204600F054FA01222046BDE8C3
:100800001040402100F04DBA01221021204600F096
:1008100048FA0022E1E701221021204600F041FAC7
:100820000022E6E710BD00000010024070B5012272
:10083000084D14022146284600F033FA00222146D2
:10084000284600F02EFA21462846BDE870400122D5
:1008500000F027BA00040240FEE7002070470000C5
:1008600010B50B4C42F220012088B0EBE10209D018
:10087000A0F51052243A04D1064800F03FF80420B5
:10088000208010BD044800F039F842F22400F7E758
:1008900006010020203E0020001E0020002070479E
:1008A00010B500220449054802F02EFB0449034814
:1008B00002F01DFB002010BDD40E0020F801002026
:1008C000D406002010B504460146084802F00FFB8C
:1008D000064802F0E5FA0648216801606168416057
:1008E000044901200870002010BD0000F80100201C
:1008F000170100201F01002000207047094A10B591
:10090000D2F8BC22D2F814220AB1012010BD0A4646
:100910000146044802F0F8FABDE81040014802F030
:100920006DBB0000F8010020F0B54048002501260D
:10093000057045708570C57080F8046480F80564A2
:1009400080F8066480F80764022780F8087880F849
:10095000097880F80A7880F80B784FF0030C80F85B
:100960000CCC80F80DCC80F80ECC80F80FCC042194
:1009700000F580500522017441748174C17480F8BF
:10098000142480F8152480F81624062380F81724F0
:1009900080F8183880F8193880F81A3880F81B3831
:1009A000072480F81C4C80F81D4C80F81E4C80F801
:1009B0001F4C00F58150057045708570C57080F83A
:1009C000046480F8056480F8066480F8076480F8A1
:1009D000087880F8097880F80A7880F80B7880F831
:1009E0000CCC80F80DCC80F80ECC80F80FCC1048E1
:1009F000017041708170C17080F8042480F8052472
:100A000080F8062480F8072480F8083880F8093830
:100A100080F80A3880F80B3880F80C4C80F80D4CC0
:100A200080F80E4C80F80F4CF0BD0000001E002036
:100A3000304E00207047012000F02AB8042000F05A
:100A400027B8082000F024B8102000F021B872B6B2
:100A5000FEE7000070B5044600F028F90546601C6A
:100A600002D004480078044400F020F9401BA04262
:100A7000FAD370BD64000020042806D10348017831
:100A8000012902D14168491C4160704720010020C2
:100A9000044910B50A68024202D00860FFF7ECFF73
:100AA00010BD0000143C01402DE9F84FDFF8BCA157
:100AB0000022012503264FF00F090AF1040BAAF1C9
:100AC000040E00BF0B6805FA02F42340A34270D164
:100AD0000F7907F00307012F01D0022F16D1876885
:100AE0004FEA420806FA08FC27EA0C07D1F80CC0C6
:100AF0000CFA08FC4CEA070CC0F808C04768A7438A
:100B00000C79C4F3001494403C4344600C79E443F2
:100B1000A4070AD0C4684FEA420C06FA0CF7BC439B
:100B20008F6807FA0CF72743C7600C7904F00304B9
:100B3000022C12D1D40800EB840CDCF820405707BB
:100B4000FF0E09FA07F824EA0804D1F8108008FA21
:100B500007F848EA0408CCF8208004684FEA420C01
:100B600006FA0CF7BC430F7907F0030707FA0CF7F6
:100B7000274307604C6814F4403F70D03C4C276812
:100B800047F480472760246822F0030704F4804478
:100B90000094384C07EB040CDCF8084897074FEA40
:100BA000177809FA08F7BC43334FB84202D100273F
:100BB00024E054E0314FB84201D101271EE0304F0C
:100BC000B84201D1022719E02E4FB84201D10327C4
:100BD00014E02D4FB84201D104270FE02B4FB8424B
:100BE00001D105270AE02A4FB84201D1062705E0C6
:100BF000284FB84201D1072700E0082707FA08F775
:100C00002743CCF80878DAF800405746D1F804C0FA
:100C10009C435FEACC2C00D51C433C60DBF80040D1
:100C20005F46D1F804C09C435FEA8C2C00D51C437E
:100C30003C60DEF800407746D1F804C09C435FEA90
:100C40008C3C00D51C433C60084F083F3C68D1F801
:100C500004C09C435FEACC3C00D51C433C60521C62
:100C6000102AFFF42FAFBDE8F88F0000083C0140C8
:100C700044380240003001400000024000040240BD
:100C800000080240000C0240001002400014024024
:100C900000180240001C02400069084000D00120FA
:100CA00070470AB1816170470904FBE70148806819
:100CB00070470000640000200248816802781144F7
:100CC00081607047640000200B4810B5016841F452
:100CD00000710160016841F480610160016841F4C4
:100CE00080710160032000F06FF80F2000F006F81B
:100CF00000F024F8002010BD003C024070B50D4DFE
:100D000004464FF47A712878B1FBF0F00A4909687B
:100D1000B1FBF0F001F074F848B9102C07D20022B2
:100D20002146501E00F030F800206C6070BD01209C
:100D300070BD000064000020700000200A4808B563
:100D4000016841F480410160006800F48040009037
:100D50000548001F016841F080510160006800F003
:100D60008050009008BD000044380240002809DB94
:100D700000F01F02012191404009800000F1E020B5
:100D8000C0F8001170470000F0B40E4B1B680C4611
:100D9000C3F30223C3F10705042D00D90425191D4F
:100DA000072901D2002300E0DB1E012606FA05F127
:100DB000491E214099409E40761E16403143F0BCAA
:100DC00003F0A3BC0CED00E0064900F00702086840
:100DD0004FF6FF03184040EA0220034A1043086020
:100DE000704700000CED00E00000FA057047006855
:100DF000416200207047F0B50368586A39B19C6AB7
:100E00004FF4827600EB144400204D1E0AE040EAC5
:100E1000024098620FE006EB8007DF59401C04EBAC
:100E20001744C0B2A842F6D344EA02404FF480729D
:100E300002EB810158500020F0BDD0F8080502F007
:100E400062BB01EBC10200EB8202D0F80805D26C54
:100E500002F0B7BA01EBC10200EB8202D0F808053C
:100E6000D2F88C2202F008BBD0F8080502F04DBB86
:100E70000A0601F00F0101EBC10100EB810101D570
:100E80003C3101E001F51F71006803F085BA70B5CF
:100E900004460B0601F00F0000EBC00104EB8101DA
:100EA0004FF001024FF0000503D581F83D203C31A1
:100EB00003E081F87D5201F51F71087094F8BC04BD
:100EC000012808D084F8BC24206802F01FFF84F8B1
:100ED000BC54002070BD022070BD70B5044601F006
:100EE0000F006268904201D9012070BD0B0601F02D
:100EF0000F0101EBC10104EB81014FF001024FF042
:100F0000000503D581F83D203C3103E081F87D5296
:100F100001F51F718D70087094F8BC04012808D089
:100F200084F8BC24206803F0EDF884F8BC54002059
:100F300070BD022070BD01F00F0101EBC10100EB9B
:100F40008100D0F89C0270472DE9F04104460F065D
:100F500001F00F0000EBC00104EB81014FF001062E
:100F60004FF0000503D581F83D603C3103E081F886
:100F70007D5201F51F710870CA600B714A7802B189
:100F80000881022B00D14D7194F8BC04012809D0CE
:100F900084F8BC64206802F011FE284684F8BC5432
:100FA000BDE8F0810220FBE770B50C4601F00F05AB
:100FB00005EBC50100EB8101C1F89432C1F88C2228
:100FC0000023C1F89C3281F87D3281F87C5203699C
:100FD00001F51F71012B00D14A612207027C0068D4
:100FE00003D003F0E7F8002070BD02F0D1FFFAE76C
:100FF00070B504460D4601F00F006168884201D9C2
:10100000012070BD29064FF000064FF0010207D500
:1010100000EBC00104EB810181F83D203C3107E089
:1010200005EBC50104EB810181F87D6201F51F71BB
:101030008A70087094F8BC04012807D084F8BC2496
:10104000206803F08BF8280702D007E0022070BD6B
:10105000217C04F2C442206803F028F884F8BC64C0
:10106000002070BD70B50C4601F00F0505EBC50101
:1010700000EB81014B65CA640023CB65012381F835
:101080003D3001F83C5F0369012B00D14A61220722
:10109000027C006803D003F08DF8002070BD02F0E0
:1010A00077FFFAE72DE9FC5F05680446284603F060
:1010B00014FA00287DD1206803F03BFA002878D08C
:1010C000D5F80808C0F30D20C4F8FC04206803F02C
:1010D00030FA800704D52068416901F002014161BE
:1010E000206803F026FAC10604F2C440009034D50B
:1010F0002068816921F0100181612F6A07F00F00DB
:1011000000EBC00004EB8006C7F3434006F51F76F2
:10111000022802D0062811D01AE047F6F0700742E4
:1011200016D0C7F30A1217462846316903F005FAAC
:10113000306938443061306A384408E00822284673
:10114000009903F0FAF9306AC7F30A1108443062D3
:101150002068816941F010018161206803F0E9F99C
:1011600000034FF0080B4FF0000A4FF001097CD547
:101170000026206803F0BCF9074674E0F80770D039
:10118000F1B2206803F0CDF98046C00707D005EB27
:101190004611C1F8089B3146204601F065FA5FEA26
:1011A000087024D505EB4611C1F808BB2068016C16
:1011B00000E025E200EB46100191D0F8082BFC4B33
:1011C000994205D9110403D54FF40041C0F8081B1A
:1011D000204600F02FFBF6490198884207D9206984
:1011E000012804D120680121009A02F05FFF5FEA24
:1011F000C86004D505EB46111020C1F8080B5FEA62
:1012000088701DD56869000605D5D5F8040840F436
:101210008061C5F8041806EBC60004EB800090F866
:101220007F1200F51F70012905D180F803A0F1B2EB
:10123000204600F0EBF905EB46110220C1F8080B3F
:101240005FEA886004D505EB46102021C0F8081B32
:101250005FEA884005D505EB46104FF40051C0F811
:10126000081B7F08761C002F88D1206803F061F9E5
:1012700040036FD5206803F034F90746002667E085
:10128000F80763D0F1B2206803F039F98046C0074F
:1012900023D006F00F0209FA02F0D5F83428824371
:1012A000C5F8342805EB4610C0F8089920690128D4
:1012B0000FD106EBC60004EB8000D0E912211144E7
:1012C000C16436B9606D20B920680121009A02F02E
:1012D000EDFEF1B22046FFF7B4FD5FEA087003D5DA
:1012E00005EB4611C1F808B95FEAC86004D505EB03
:1012F00046111020C1F808095FEA486004D505EBE3
:1013000046104021C0F808195FEA887017D53146A9
:10131000284603F0B5F806EBC60004EB800090F811
:101320003F103C30012905D180F803A0F1B22046DE
:1013300000F068F905EB46110220C1F808095FEAE0
:10134000086003D53146204601F0F4F97F08761C89
:10135000002F95D1206803F0ECF8002811DAD5F8B9
:10136000040820F00101C5F8041894F8F4040128D9
:101370002BD0204600F042FA2068416901F000417C
:101380004161206803F0D5F800050BD5D5F80808B1
:10139000C00702D0204600F075FA2068416901F4C8
:1013A00000614161206803F0C4F8C00466D5D5F837
:1013B000040820F00100C5F804081021206803F09B
:1013C0005FF800214FF67F321FE084F8F4A400217B
:1013D0002046FFF70BFDCFE705EB4110C0F80829C9
:1013E000D0F8003923F40013C0F80039C0F8082BF6
:1013F000D0F8003B23F40013C0F8003BD0F8003BCA
:1014000043F00063C0F8003B491C60688842E3D8A1
:10141000D5F81C0840F00111C5F81C18206B0028F5
:1014200028460DD0D0F8840840F00B01C5F8841888
:10143000D5F8440840F00B012846C5F844180DE0E3
:10144000D0F8140842F22B010843C5F81408D5F867
:10145000100840F00B012846C5F81018D0F8000815
:1014600020F4FE61C5F80018217C2068009A02F083
:101470001DFE2068416901F480514161206803F03C
:1014800058F8800415D5206802F0D8FB206803F0D6
:1014900017F8E06000F0A8FA0146227B206803F00C
:1014A000ABF8204600F094F92068416901F400513E
:1014B0004161206803F03DF8000707D5204600F0A1
:1014C000A1F92068416901F008014161206803F039
:1014D00030F8000616D5A86920F08000A861012622
:1014E0000DE000BF06EBC60004EB800090F87F0221
:1014F000012803D1F1B22046FFF7BAFC761C6068E0
:10150000B042EFD8206803F014F8C00221D50126BC
:101510004F4616E005EB4610D0F8001906EBC60062
:1015200004EB800090F84020012A09D1002907DA55
:1015300080F83F70F0B240F080012046FFF798FC41
:10154000761C6068B042E5D82068416901F48011DA
:101550004161206802F0EDFF800234D501204B4646
:1015600029E000BF05EB4011D1F8001B00EBC002E1
:1015700004EB820696F88022012A1BD1002919DA91
:1015800094F8FC2401F4803102F00102914211D15F
:1015900086F87F32A96941F08002AA61696909066B
:1015A00008D4D5F8040840F40070C5F8040805E034
:1015B0000A30544F401C61688142D3D82068416989
:1015C00001F400114161206802F0B3FF400007D52B
:1015D0002046FFF732FC2068416901F080414161FB
:1015E000206802F0A6FF40070AD520684568680712
:1015F00002D52046FFF738FC206841682943416046
:10160000BDE8FC9FD0F8080501F0D6BFD0F808056A
:1016100001F0E6BF2DE9F0418AB0040005D094F84E
:10162000BD042668002520B108E001200AB0BDE80D
:10163000F08184F8BC54204600F05EF8032084F862
:10164000BD04F06BC00500D42561206802F09AFC4F
:1016500004F11001282288466846FEF77DFE94E8D2
:101660000F0002F0F9FA0226C8BB0021206802F040
:1016700083FF002001270EE000EBC00104EB810195
:1016800081F83D7001F83C0F08810D71CD600D614E
:10169000401CC0B28D6161688142EDD8002011E02C
:1016A00000EBC00104EB810181F87D5281F87C02DE
:1016B00081F88052C1F88852C1F88C52401CC0B2E7
:1016C000C1F8945261688142EAD8282241466846AE
:1016D000FEF742FE94E80F0002F09AFB10B184F886
:1016E000BD64A2E784F8385084F8BD74206802F025
:1016F00081FB00209AE700002DE9F04186B0044606
:1017000014216846FEF75AFE2C492068884251D1C0
:101710002B4C4FF00008206840F004002060206847
:1017200000F004000590206840F00100206020686F
:1017300000F001000590206840F002002060206861
:10174000022500F0020005900D208DE821010326FE
:101750000A2769461B48CDE90367FFF7A5F928204A
:101760008DE8210169461848CDE90367FFF79CF928
:1017700043F623408DE8210169461448CDE903670B
:10178000FFF792F9206840F000502060206800F0D8
:1017900000500590206840F08040206020680022C2
:1017A00000F08040059001214D20FFF7EDFA4D201B
:1017B000FFF7DCFA06B0BDE8F0810000000004404D
:1017C000303802400008024000000240000402409D
:1017D00070B50446C068012570B1022801D0FFF73A
:1017E00036F92946D4F8080501F068FFD4F8080551
:1017F000BDE8704001F01DBF0025F2E7D0F80805F4
:1018000001F045BFD0F8080501F04BBF10B5044604
:1018100090F8BC0401280BD0012084F8BC0484F8A3
:101820003810206802F0D6FE002084F8BC0410BDF9
:10183000022010BDD0F8082500F2C441104601F086
:1018400049BF10B50446006894F8BC14012906D0BD
:10185000012184F8BC14A16A012902D008E0022009
:1018600010BDA169012903D0816B41F480318163EE
:10187000206802F0E0FD206802F0AEFA002084F853
:10188000BC0410BD10B50446D0F8080501F064FF93
:101890002068D0F8001E41F00101C0F8001E206A47
:1018A000002804D00248016841F00601016010BD23
:1018B00010ED00E02DE9F0470E46050065D0DFF899
:1018C0001481D8F80000F7B200F00700B04207D248
:1018D00088F80070D8F8000000F00700B04254D13A
:1018E00028683D4C810712D5400703D5206840F495
:1018F000E05020602878000703D5206840F460405D
:1019000020602068A96820F0F00008432060287853
:10191000C0072DD0304968680839012812D0022844
:1019200013D0032811D00968890700292DDA21680E
:1019300021F0030101432160FFF7B8F9814641F22C
:10194000883A0EE009688903EFE709688901ECE746
:10195000FFF7ACF9A0EB0901514502D90320BDE81E
:10196000F0872068696800F00C00B0EB810FEFD1C0
:10197000D8F80010404601F00701B14207D90770BE
:10198000006800F00700B04201D00120E7E72878A6
:10199000400705D52068E96820F4E050084320603E
:1019A0002878000706D52068296920F4604040EABD
:1019B000C100206000F03EF82168084AC1F303111D
:1019C000515CC8400649086006480068FFF796F970
:1019D0000020C4E7003C024008380240C24700082B
:1019E0007000002068000020014800687047000077
:1019F000700000200448054900680968044AC1F3E2
:101A00008221515CC84070477000002008380240B5
:101A1000D24700080448054900680968044AC1F330
:101A20004231515CC84070477000002008380240C5
:101A3000D2470008154810B5006810F00C02144891
:101A400013D04110042A0FD0082A0ED10F4C241FA6
:101A50002268236802F03F025B0207D52068C0F3CA
:101A60008810A0FB010106E0084610BD2168C1F303
:101A70008811A1FB00010023FEF7F7FB2168C1F3E9
:101A80000141491C4900B0FBF1F010BD083802408B
:101A90000024F4002DE9F84F04006ED02078DFF820
:101AA0004C93C007A9F104054AD009F1040001686C
:101AB000C1F38101012908D00068C0F38100022828
:101AC0000AD1D9F80000400206D52868800337D52E
:101AD00060680028E1D033E06068B0F5803F10D046
:101AE000B0F5A02F286810D020F480302860286836
:101AF00020F4802028606068A8B1FFF7D7F8064678
:101B00000DE0286840F48030F4E740F4802028603D
:101B1000F7E700BFFFF7CAF8801B642873D828686E
:101B20008003F7D50CE0FFF7C1F8064605E000BFDB
:101B3000FFF7BCF8801B6428F0D828688003F7D42E
:101B40002078DFF8AC8280074FF0000A3ED5A74826
:101B5000001D016811F00C0F08D00068C0F381006F
:101B600002280BD1D9F80000400207D4286880076A
:101B700016D5E068012800D112E033E1E068B8B181
:101B80000120C8F80000FFF791F8064605E000BF05
:101B9000FFF78CF8801B0228C0D828688007F7D58B
:101BA0002868216920F0F80040EAC10028600DE0B3
:101BB000C8F800A0FFF77AF8064604E0FFF776F8C9
:101BC000801B02281FD828688007F7D420780007D8
:101BD00022D5864F87486169703771B10121016054
:101BE000FFF764F8064604E0FFF760F8801B022860
:101BF00009D838688007F7D50EE0C0F800A0FFF7D5
:101C000055F8064605E082E0FFF750F8801B0228F1
:101C10007DD838688007F7D42078400768D5DFF88A
:101C2000CCB100270BF13C0BDBF80000C0000BD45B
:101C3000DBF8001041F08051CBF80010DBF8000019
:101C4000012700F0805000906B4E3068C00510D422
:101C5000306840F480703060FFF728F8009005E0AD
:101C6000FFF724F80099401A022850D83068C005C0
:101C7000F6D55E4EA0686C3601280FD00528306876
:101C800010D020F001003060306820F00400306097
:101C9000A068B8B1FFF70AF800900FE0306840F094
:101CA0000100F4E740F004003060F7E7FEF7FEFFC4
:101CB0000099411A41F28830814266D83068800725
:101CC000F4D50EE0FEF7F2FF009007E0FEF7EEFF1E
:101CD0000099411A41F28830814256D83068800715
:101CE000F4D42FB1DBF8001021F08051CBF80010B4
:101CF000A069C8B33D49091D0968C1F381010229E2
:101D00004AD00228504607D0C8F8600000E03CE006
:101D1000FEF7CCFF04463BE04746C8F86000FEF7FC
:101D2000C5FF064605E000BFFEF7C0FF801B022886
:101D30002BD828688001F7D4D4E907010843A16AA9
:101D40002E4A490802EB0141626A41EA82110843C6
:101D500094F82C1040EA0161C9F80010012038669F
:101D6000FEF7A4FF044606E03EE000BFFEF79EFF3C
:101D7000001B022809D828688001F7D534E000BF8D
:101D8000FEF794FF001B022802D90320BDE8F88F5C
:101D900028688001F4D427E00128F7D0D9F80000A2
:101DA000E26900F4800191421CD1226A00F03F01F7
:101DB000914217D147F6C071626A0140B1EB821FB0
:101DC00010D1A26A4FF0FF3300F4403103EB52020E
:101DD000B1EB024F06D194F82C1000F07060B0EB1C
:101DE000016F01D00120D1E70020CFE70438024085
:101DF00000004742800E4742007000400000FFFF95
:101E000010B5401EB0F1807F01D3012010BD4FF00E
:101E1000E02460610F21601702F077FC0020A061D0
:101E200007202061002010BD7047704770B590F802
:101E30003C20012A32D0012480F83C40022280F864
:101E40003D2003685A689D6822F070060A68324394
:101E50005A60134B02689A4214D0B2F1804F11D0ED
:101E6000104B9A420ED0104B9A420BD00F4B9A4215
:101E700008D00F4B9A4205D00E4B9A4202D00E4B1F
:101E80009A4204D1496825F080031943916080F893
:101E90003D40002180F83C10084670BD022070BD16
:101EA000000001400004004000080040000C004019
:101EB00000040140004001400018004010B504003B
:101EC00003D094F83D0010B107E0012010BD0020C0
:101ED00084F83C00204600F01FF8022084F83D0002
:101EE000211D206800F010FD012084F8460084F8D0
:101EF0003E0084F83F0084F8400084F8410084F8F4
:101F0000420084F8430084F8440084F8450084F8D3
:101F10003D00002010BD000008B500680B49884254
:101F200012D10B48016841F00201016000680322F0
:101F300000F00200009011461D20FEF725FFBDE8CD
:101F400008401D20FEF712BF08BD0000000400403D
:101F50004038024090F83D10012901D0012070471F
:101F6000022180F83D100168CA6842F00102CA608F
:101F700000681149884214D0B0F1804F11D00F4948
:101F800088420ED00E4988420BD00E49884208D0B4
:101F90000D49884205D00D49884202D00C4988423B
:101FA00004D1816801F00701062903D0016841F0DE
:101FB0000101016000207047000001400004004062
:101FC00000080040000C00400004014000400140B7
:101FD0000018004070B5044690F83C000025012828
:101FE00017D0012684F83C60022084F83D00206868
:101FF000826822F0770222F47F42826008685028CB
:1020000038D00DDC20284FD005DC90B3102811D13A
:102010004AE0022070BD302846D040280AD13BE07B
:1020200060282FD070280DD0B0F5805F03D0B0F5B8
:10203000005F12D0012584F83D60002084F83C0048
:10204000284670BDCB68D1E90121206800F0C0FCB2
:102050002068816841F0770109E0CB68D1E901216E
:10206000206800F0B5FC2068816841F480418160FF
:10207000E1E719E0CA684968206800F0BBFC50211C
:10208000206806E0CA684968206800F0C4FC602146
:10209000206800F0A7FCCEE7CA684968206800F015
:1020A000A9FC40212068F4E7226801461046F0E7C9
:1020B000704770B50446006801694FF00005C943D8
:1020C000890715D4C168C943890711D4E91E016184
:1020D00001202077206880698007204602D0FFF722
:1020E000E7FF04E000F098F8204600F096F8257726
:1020F00020680169C943490717D4C168C943490722
:1021000013D46FF0040101610220207720688069F8
:1021100010F4407F204602D0FFF7CAFF04E000F031
:102120007BF8204600F079F8257720680169C943DB
:10213000090716D4C168C943090712D46FF0080112
:102140000161042020772068C0698007204602D002
:10215000FFF7AEFF04E000F05FF8204600F05DF806
:10216000257720680169C943C90617D4C168C943E6
:10217000C90613D46FF01001016108202077206890
:10218000C06910F4407F204602D0FFF791FF04E0C1
:1021900000F042F8204600F040F8257720680169F9
:1021A000C943C90708D1C168C943C90704D1891EF9
:1021B0000161204600F032F820680169C943090630
:1021C00009D4C168C943090605D46FF080010161D3
:1021D0002046FFF729FE20680169C943490609D452
:1021E000C168C943490605D46FF04001016120462A
:1021F00000F03AF820680169C94389060BD4C16828
:10220000C943890607D46FF0200101612046BDE86B
:102210007040FFF70ABE70BD7047704770B50D493A
:10222000884215D10C4C0D4D00262088401C80B2F0
:102230002080297801290AD109490988884207D1D3
:102240000848FEF743FA26802878012800D0268027
:1022500070BD0000280100200A01002004010020B8
:102260000C010020001E0020704770B5040004D04F
:1022700094F83D00002510B106E0012070BD84F8FF
:102280003C50204600F022F8242084F83D002068CD
:10229000C16821F40051C160204600F0CFFB2068E6
:1022A000016921F4904101612068416921F02A010E
:1022B00041612068C16841F40051C160256420205B
:1022C00084F83D0084F83E00002070BD70B586B0F3
:1022D000044614216846FEF771F8234E2268002157
:1022E0002248022303240725B2421AD11F4A14327E
:1022F000166846F010061660126802F01002059289
:10230000026842F002020260006802AA00F00200C5
:10231000059082E83200C020CDE9000369461448E8
:102320001DE0144EB2421CD1104A1032166846F419
:1023300080261660126802F480220592026842F03C
:1023400004020260006802AA00F00400059082E81E
:1023500032004FF44060CDE9000369460648FEF7BD
:10236000A3FB06B070BD00000010014030380240F1
:10237000000402400048004000080240FEE7000060
:1023800030B51948034604785A789978DB78002CE0
:1023900021D0012C1FD1012A1DD101291BD1012BD4
:1023A00019D1014605794B790024C11E15B1012DC3
:1023B00003D005E023B94C7002E0012B00D14A7034
:1023C00083790948C0793BB1012B09D0022B02D196
:1023D000022800D1087030BD0028FCD10C7030BD3F
:1023E0000128FCD10A7030BD17010020F0B5002390
:1023F0000A24302537261F4611E000BFB4EB107FBA
:1024000002D905EB107C01E006EB107C01F813C04B
:1024100001EB430C00015B1C8CF80170DBB29342B2
:10242000ECD3F0BDF0B587B014216846FDF7C6FFC8
:102430003A48016841F004010160016801F00401BB
:102440000591016841F080010160016801F080019F
:102450000591016841F001010160016801F001018D
:102460000591016841F002010160016801F002017B
:102470000591016841F008010160016801F008015F
:102480000591016841F0200101600068012200F01F
:102490002000234E1403059021463046FEF701FC30
:1024A000204F012208213846FEF7FBFB009401244F
:1024B0000225694630460194CDE90245FEF7F4FA5B
:1024C0000820CDE9000469463846CDE90245FEF70B
:1024D000EBFA042000904FF48810CDE9010569461D
:1024E0001148FEF7E1FA002205210820FEF74CFC16
:1024F00001220E4F560231463846FEF7D2FBCDE997
:10250000006469463846CDE90245FEF7CDFA01225E
:1025100031463846FEF7C5FB07B0F0BD3038024003
:1025200000080240000C024000000240001402407B
:1025300010B586B0002416480094019402940394C8
:1025400004941249059401605321C0E90114182133
:10255000C0E903148461FFF7B1FC08B1FEF777FA14
:102560004FF48050009069460948FFF733FD08B1E9
:10257000FEF76DFA049404A905480594FFF756FC8C
:10258000002801D0FEF763FA06B010BD0004004039
:10259000280100200C4810B50A4901604FF4E131D0
:1025A0004160002181600C22C160C0E90412816198
:1025B000C161FFF75AFE002803D0BDE81040FEF7C6
:1025C00046BA10BD00100140700100200C4810B543
:1025D0000A4901604FF4E1314160002181600C2221
:1025E000C160C0E904128161C161FFF73EFE0028AD
:1025F00003D0BDE81040FEF72ABA10BD00480040E5
:10260000B401002010B501220F49104800F0B4FEBB
:1026100008B1FEF71CFA0E490C4801F0C5F808B1E4
:10262000FEF715FA0B49094800F056FC08B1FEF711
:102630000EFA064801F03CF9002803D0BDE810402E
:10264000FEF705BA10BD000000000020F8010020D0
:10265000CC00002050000020FEE7FEE70148FEF716
:1026600021BD0000F41800202DE9F04103680D465B
:1026700004461E6C03EB4511D1F8080BD4F810E0AA
:102680004FF400474FF0200C04F2C442BEF1010F9A
:1026900009D0DFF898E0764539D1020432D500BF81
:1026A000C1F8087B3FE0224B5FEA007E04D59E42E2
:1026B00039D90004F4D436E05FEA806E02D5C1F85F
:1026C00008CB30E010F0280F2DD19E4201D9000434
:1026D000E6D405EBC50004EB8000D1F8101BD0F860
:1026E0009832C1F31201591AC0F89C1200F51F70FC
:1026F000ADB983691BB10269114401610FE0012189
:1027000020680AE080060AD5C1F808CB07E035B991
:10271000D4F8940218B90021184601F0C7FCE9B2B8
:102720002046FEF797FB0020BDE8F0810A31544FA8
:102730000A30544F2DE9F84F0E4601EBC60100EB6D
:10274000810481460568616DE06D3C34884202D9A0
:102750000120BDE8F88F081AE168814200D20846DE
:10276000C01C870805EB46181BE000BFA0EB010A60
:10277000E068504500D282460AF10300870899F8C4
:10278000100000901FFA8AF3F2B22846216901F086
:10279000A7FF216901EB0A002061216A01EB0A0011
:1027A0002062D8F8180980B2B84205D3216AA0691E
:1027B000814201D20028D9D1216AA069884208D873
:1027C00006F00F0101208840D5F834188143C5F880
:1027D00034180020BDE7704770470178407841EA1F
:1027E000002070471649174A01200B7823B1012BAE
:1027F00004D0022B06D103E0108003E0022300E0A6
:10280000042313804A78104B012A01D012B103E04F
:10281000187001E000221A70897801290ED180F326
:102820001388BFF34F8F09480168094A01F4E0613A
:1028300011430160BFF34F8F00BFFDE770470000F9
:10284000140100200C010020040100200CED00E028
:102850000400FA05FEF730BA30B593B0302168466F
:10286000FDF7ACFD14210CA8FDF7A8FD1D480025BF
:10287000016841F080510160006800F080501190C3
:102880001948016841F4804101600068022400F4A5
:102890008040119001200090000401908001CDE95A
:1028A000064008AA0420A82182E813000B9068467D
:1028B000FFF7F0F808B172B6FEE70CA90F2081E827
:1028C00031004FF4A0500F904FF48050109005212C
:1028D0000CA8FEF7EFFF002801D072B6FEE713B098
:1028E00030BD0000403802400070004002480168DE
:1028F00041F470010160704788ED00E00148FFF786
:10290000D8BB000028010020F0B50268254C264DF8
:10291000264E274F274B4FF0804CA04209D06045F0
:1029200007D0A84205D0B04203D0B84201D09842A7
:1029300004D122F0700E4A6842EA0E02A0421BD077
:10294000604519D0A84217D0B04215D0B84213D074
:10295000984211D0184DA8420ED0184DA8420BD065
:10296000174DA84208D0174DA84205D0164DA842D1
:1029700002D0164DA84203D122F44075CA682A43FA
:102980004D6922F080022A4302608A68C2620A68A6
:102990008262A04201D0984201D1096901630121FC
:1029A0004161F0BD0000014000040040000800400B
:1029B000000C004000040140004001400044014080
:1029C0000048014000180040001C0040002000406A
:1029D00010B5846842EA032224F47F440A43224368
:1029E000826010BD826822F070020A4342F0070143
:1029F0008160704710B5036A046A24F00104046220
:102A0000846924F0F00444EA021423F00A020A4321
:102A10008461026210BD10B5036A23F010030362E3
:102A20008369046A23F4704343EA023224F0A0036A
:102A300043EA01118261016210BD000070B50446D5
:102A400000680169E26821F4405111430161216984
:102A5000A068E26908436169114308432168CA68B4
:102A600049F20C639A430243CA6020684169A26933
:102A700021F440711143416131492068884202D0FC
:102A80003049884202D1FEF7C5FF01E0FEF7B2FFF0
:102A9000E2690023192164253226B2F5004F6268ED
:102AA00028D0A0FB0101930F9200FDF7DEFB014649
:102AB000B0FBF5F06FF01802504301EB800006EB1D
:102AC0000010B0FBF5F000F0F002B1FBF5F002EB06
:102AD0000012B1FBF5F06FF01803584301EB8000D2
:102AE00006EB0010B0FBF5F000F00F002168104479
:102AF000886070BDA0FB010192185B41FDF7B5FB3A
:102B00000146B0FBF5F00201B1FBF5F06FF01803E0
:102B1000584301EB800006EBC000B0FBF5F000F07D
:102B2000F80002EB4002B1FBF5F0584301EB8000E6
:102B300006EBC000B0FBF5F000F00700D6E70000A0
:102B400000100140001401402DE9F0410C46D0F87E
:102B5000D412D0F8C82200EB8101D1F8C01229B3F9
:102B600004F00F0606EB860300EB83050027AB6934
:102B70004BB106EBC60602EB8602926CB3FBF2F693
:102B800002FB1632A2B1C1F81472D0F8D42200EBC5
:102B90008200D0F8C40203692BB1D1F808022246A2
:102BA00001F5047198470020BDE8F0810320FBE7A0
:102BB00000231A462146AF6100F0D7FDF3E770B558
:102BC0000546D0F8D40205EB8000D0F8C04294B19D
:102BD000284600F0A9FCC4F80C02D5F8D412D4F8A9
:102BE000040205EB8101D1F8C412CA6804F503712F
:102BF0009047002070BD032070BD000070B5224DCD
:102C00000446297800F0D4FB2878002600F00F0055
:102C100000EB800004EB800086846978204600F099
:102C2000C7FB687800F00F0000EB800004EB800029
:102C3000A0F86461A978204600F0BAFBA87800F0FB
:102C40000F0000EB800004EB80008684C684D4F87B
:102C5000D40204EB8000D0F8C01299B1D0F8C402BD
:102C600040688047D4F8D40204EB8000D0F8C0025A
:102C700000F09FFFD4F8D40204EB8000C0F8C062DB
:102C8000C4F8BC62002070BD7800002010B5D0F8F8
:102C9000D41200EB8100D0F8C04284B1D0F8C41245
:102CA00059B194F80002FF2807D08B6894F80122EC
:102CB00021469847FF2084F80002002010BD032021
:102CC00010BD00000A210180004870477C000020F0
:102CD00070B5064682210C4800F086FA05460121AF
:102CE000094800F081FA04468121074800F07CFA87
:102CF0000DB11021A971402104B1A18000B18180E2
:102D000043203080004870BD8800002070B5064622
:102D100082210D4800F068FA054601210A4800F0BA
:102D200063FA04468121084800F05EFA0DB11021D3
:102D3000A9714FF4007104B1A18000B181804320DA
:102D40003080014870BD00008800002070B5064644
:102D500082210C4800F048FA05460121094800F09C
:102D600043FA04468121074800F03EFA0DB11021D4
:102D7000A971402104B1A18000B18180432030803D
:102D8000004870BD880000202DE9F04704464FF44C
:102D90000775284600F00EFF06004FF0000863D0CC
:102DA0002946FDF70BFBD4F8D4023C4D04EB800020
:102DB0004FF01009C0F8C062C4F8BC62207C4FF428
:102DC000007A0127F0B3402302222978204600F040
:102DD0001BFC2878402300F00F0000EB800004EB80
:102DE0008000878402226978204600F00DFC687814
:102DF000082300F00F0000EB800004EB80000322AA
:102E0000A0F86471A978204601F00F0101EB81015F
:102E100004EB8101A1F82690A97800F0F5FBA878D1
:102E200000F00F0000EB800004EB80008784C6F800
:102E30000482D4F8D402474604EB8000D0F8C402E0
:102E4000006800E018E006F5017680473761776199
:102E500032687AB1207CF8B140236978204600F0CE
:102E6000DFFB0020BDE8F087D4F8D41204EB810129
:102E7000C1F8C0820220F5E7534602222978204695
:102E800000F0C2FB2878534600F00F0000EB8000F2
:102E900004EB80008784A5E75346DEE77800002036
:102EA00010B5D0F8D41200EB8101D1F8C01259B19D
:102EB000027C084C002AD1F8042207D04023617814
:102EC00000F0AEFB002010BD032010BD4FF40073D6
:102ED000F5E700007800002039B1D0F8D42200EBEB
:102EE0008200C0F8C4120020704703207047D0F859
:102EF000D42200EB8200D0F8C00218B1C0F804124E
:102F00000020704703207047D0F8D43200EB8300D4
:102F1000D0F8C00228B1C0F81022C0F80812002072
:102F20007047032070472DE9FC410646D0F8D402D3
:102F30000C4606EB80000021D0F8C0728DF800101E
:102F4000ADF804100D4637B1217811F060022FD092
:102F5000202A4BD102E00320BDE8FC81E288F2B1D7
:102F600009060DD5D0F8C40263783946D0F808C0F8
:102F70001846E047E288072A00D9072239462DE0A3
:102F8000607887F80002E088402800D34020C2B271
:102F900087F801223946304600F081F82BE0D0F85E
:102FA000C40263780022866821461846B04722E0B2
:102FB000607830B101281ED00A2809D00B2815D11D
:102FC00010E096F89C02032810D1022201A905E026
:102FD00096F89C02032809D101226946304600F088
:102FE00078F808E096F89C02032804D02146304681
:102FF00000F04AF803252846AEE7000010B5D0F8E7
:10300000D41200EB8101D1F8C02201211AB1D2F80B
:10301000143213B116E0032010BD0121C2F81412BE
:103020000949D2F81032097801F00F0404EB840446
:1030300000EB8404A361D2F81032D2F8082200F029
:1030400094FB0021084610BD7800002010B5D0F890
:10305000B82200245268904700B10324204610BDD6
:103060000020704700207047134610B50A46002123
:1030700000F0D6FA002010BD134610B50A46002114
:1030800000F073FB002010BD10B50446802100F055
:1030900051FB2046BDE81040002100F04BBB10B5AD
:1030A0000323C0F89432C0F858211346C0F85C21BD
:1030B0000A46002100F0B4FA002010BD10B5052129
:1030C000C0F8941200231A46194600F0A9FA00200D
:1030D00010BD10B50223C0F8943282611346C2615C
:1030E0000A46002100F041FB002010BD10B504216C
:1030F000C0F8941200231A46194600F036FB00204F
:1031000010BDF8B504460020ADF8000048880D4613
:10311000010A08295FD2DFE801F05E0409175E5E4C
:103120003C45D4F8B412207C0A6819E0207C0226C1
:103130000028D4F8B80205D0C16A6846884701461D
:10314000467039E0816AF8E7C0B2062843D2DFE86A
:1031500000F0030A1014181CD4F8B402426805E009
:10316000694690471CE0D4F8B402826892B3207C90
:10317000F6E7D4F8B402C268F8E7D4F8B4020269FA
:10318000F4E7D4F8B4024269F0E7D4F8B4028269F3
:10319000ECE7207CF0B9D4F8B802416B6846884768
:1031A000014609E0207CA8B9D4F8B802016B684652
:1031B0008847014607204870EA888AB1BDF80000B8
:1031C00040B1824200D90246ADF800202046FFF708
:1031D00080FFF8BDFFE729462046FFF755FFF8E7D7
:1031E0002046FFF783FFF4E778B50E464288017862
:1031F000002504468A4212D9ADF800100AE069465B
:1032000000F00FF84178052904D181780546B142D4
:1032100005D000256188BDF800209142EFD82846EE
:1032200078BD0A8803781A440A80017808447047F8
:1032300070B5002300281ED00025044602E06D1C56
:10324000EDB2641C2678002EF9D1022404EB45046B
:1032500014801278CA545B1C0322CA5400245B1CDD
:1032600006E0CA545B1CDAB28C54521CD3B2401C28
:103270000278002AF5D170BD01004FF0000004D0A3
:10328000012901D0022901D0032070470120704795
:1032900010B50A46024903A0FFF7CAFF004810BD57
:1032A000D404002043444320436F6E6669670000E6
:1032B00012200880004870472000002010B50A4600
:1032C000024903A0FFF7B4FF004810BDD40400205A
:1032D00043444320496E7465726661636500000073
:1032E00004200880004870471C00002010B50A46E2
:1032F000024903A0FFF79CFF004810BDD404002042
:1033000053544D6963726F656C656374726F6E6957
:103310006373000010B50A46024903A0FFF788FF57
:10332000004810BDD404002053544D333220566958
:10333000727475616C20436F6D506F727400000081
:1033400010B51A2008800A480168001D0468001D95
:103350000068081809D008220649FFF747F8054910
:10336000042210312046FFF741F80248801E10BDAC
:10337000107AFF1F3600002078B10023C0F8B83261
:10338000C0F8C432C0F8D03209B1C0F8B41201217B
:1033900080F89C12027000F0CBB80320704710B583
:1033A000D0F8C802FDF799FDBDE81040FFF764BFF3
:1033B00010B5D0F8C802FDF76AFDBDE81040FFF770
:1033C0005BBF2DE9F04117460446002521B194F872
:1033D0009C02032842D04CE0D4F8941204F114006B
:1033E000022935D1D0E902639E4206D9F21A8260E1
:1033F00039462046FFF740FE0FE0B34214D1406843
:10340000984211D3D4F8981288420DD20022114666
:103410002046FFF731FEC4F8985200231A46194699
:10342000204600F0FDF813E094F89C02032808D130
:10343000D4F8B802C16821B1C4F8D452C16820469A
:1034400088478021204600F075F92046FFF736FEB8
:1034500094F8A00268B184F8A0520AE0D4F8B80247
:10346000426932B1C4F8D4524269204690470028DC
:1034700000D10020BDE8F08170B51346044600225B
:1034800021B194F89C02032830D03AE0D4F8941289
:1034900004F5AA70032934D1D0E902518D420AD92A
:1034A0006A1A82600846824200D3024619462046C4
:1034B000FFF7DAFD25E094F8AA0210F01F0003D010
:1034C000012802D0022800D0002294F89C02032890
:1034D00008D1D4F8B802016921B1C4F8D422016935
:1034E000204688472046FFF701FE0AE0D4F8B802DC
:1034F000836933B1C4F8D4228269204690470028FA
:1035000000D1002070BD0020704710B500240121BB
:1035100080F89C12D0F8B82222B152680179904705
:1035200000B10324204610BDD0F8C802FDF703BD4A
:1035300010B50178012929D115490122C1F80805E2
:10354000C0F8C81213480860062048600020C1E98E
:103550000302C1E9062008624862C8620863486342
:103560000846FEF757F808B1FDF771FA4FF40071FD
:103570000748FDF73CFC802200210548FDF73BFC95
:103580004FF4BA7201210248FDF735FC002010BD4E
:10359000F4180020000004400A0601F07F01D0F872
:1035A000C80201EBC10100EB810002D590F83E009A
:1035B000704790F87E02704710B5D0F8D42200EB27
:1035C0008202D2F8B82222B190F89C32032B02D0AA
:1035D00004E0032010BD126A02B19047002010BD24
:1035E00010B5D0F8D42200EB8202D2F8B82222B172
:1035F00090F89C32032B02D004E0032010BD526AE5
:1036000002B19047002010BD10B51C461346D0F8FB
:10361000C8022246FDF798FCBDE81040FFF72CBE1B
:1036200010B5D0F8C802FDF7BFFCBDE81040FFF7A9
:1036300023BE2DE9F04100260125044680F89C5266
:10364000C4F894626660C4F8A46280F8A062D0F8FE
:10365000B80230B1426822B100212046904700B143
:1036600003260022402311462046FFF7CDFF4027C6
:10367000A4F864513B46002280212046C4F86071C2
:10368000FFF7C2FFA58430462762BDE8F08190F8BD
:103690009C12042903D190F89D1280F89C120020FE
:1036A000704710B590F89C12032905D1D0F8B812D4
:1036B00011B1C96901B18847002010BD0174002013
:1036C000704710B5D0F8C802FEF7A0F8BDE810406A
:1036D000FFF7D2BD70B5044600F2AA20054600F0FF
:1036E0004DF80120C4F89402B4F8B002C4F898026E
:1036F00094F8AA0210F01F010AD001290ED0022965
:1037000012D000F080012046BDE8704000F012B8F1
:1037100029462046BDE8704000F0CCB82946204636
:10372000BDE8704000F00CBA29462046BDE8704064
:1037300000F056B910B5D0F8C802FDF759FCBDE845
:103740001040FFF799BD10B5D0F8C802FEF779F820
:10375000BDE81040FFF790BD90F89C1280F89D12D4
:10376000042180F89C120020704710B5D0F8C802E0
:10377000FDF778FCBDE81040FFF77EBD70B505464B
:1037800011F8010B2870087868704C1C2046FFF770
:1037900024F86880A41C2046FFF71FF8A880A01C0E
:1037A000FFF71BF8E88070BD38B504460020ADF87F
:1037B0000000A1B1C4F8B812D4F8D40204EB800020
:1037C000D0F8B802C16A19B168468847C4F8D00277
:1037D000D4F8D802401CC4F8D802002038BD032019
:1037E00038BD02460020D2F8B832002B02D01B6848
:1037F00010461847704700002DE9F04188462B4ECF
:103800008978002504463170012906D941462046B1
:10381000FFF73AFC0320BDE8F08194F89C020227F0
:1038200002280CD003281DD041462046FFF72CFC6F
:1038300031782046FFF70AFC03252846EBE789B3D9
:1038400020466160FFF7CDFF050004D041462046C9
:10385000FFF71AFC1DE02046FFF748FC032084F820
:103860009C02EAE7C1B1606888421BD0C1B2204621
:10387000FFF7ECFB317820466160FFF7B2FF0500EF
:1038800010D041462046FFF7FFFB21792046FFF785
:10389000DDFB84F89C72D0E784F89C72204661605E
:1038A000FFF7D4FB2046FFF721FCC6E77400002099
:1038B000FFF749BF2DE9F0410A78002512F06002B8
:1038C0000CD0202A01D0402A7DD1D0F8D42200EBA0
:1038D0008202D2F8B8229268904731E04B780022F9
:1038E00001260A2B6FD2DFE803F041666E586E089E
:1038F000056E2D29FFF705FC67E004468888D8B9D6
:10390000C888C8B94888802816D200F07F0794F884
:103910009C02032810D084F89E7239462046FFF797
:10392000D0FE2046FFF7E2FB1FB1022084F89C0284
:103930004BE084F89C6248E0204644E0FFF75CFFDF
:10394000054642E0CB88012B3DD190F89C32012BFB
:1039500004D0022B02D0032B35D104E08260012277
:1039600000F1080116E00122011D13E090F89C22ED
:10397000012A03D0022A01D0032A24D1CA88022AAC
:1039800021D1C660D0F8A41209B10321C16002227E
:1039900000F10C01FFF79DFB17E04A88012A02D0D5
:1039A000022A03D00FE0C0F8A46216E08988090A51
:1039B00080F8A01211E090F89C32012B08D0022B65
:1039C00006D0032B04D0FFF75FFB2846BDE8F0814B
:1039D00049880129F9D1C0F8A422FFF787FBF4E751
:1039E0002DE9F041054608780C790E464FF00008A5
:1039F00010F060000BD0202801D040286AD1214669
:103A00002846FFF72DFBFF2800D0D8B395E070784B
:103A1000C8B3012824D003285CD195F89C02022861
:103A200002D0032856D10CE0002C53D0802C51D06A
:103A300021462846FFF77EFE80212846FFF77AFEC2
:103A40007BE0708840B93CB1802C05D0C88818B99B
:103A500021462846FFF76EFE2846FFF747FB6CE03D
:103A600095F89C020228DFD0032863D1708880BBC0
:103A7000600603D021462846FFF791FC2846FFF751
:103A800035FBBCE700E00AE0C5F8D402D5F8B8027F
:103A90008268F2B131462846904780464DE095F85D
:103AA0009C020027022802D0032843D113E00CB166
:103AB000802C3FD1200604F07F0000EB800005EB56
:103AC000800101D5143101E001F5AA7102220F60D5
:103AD0002CE032E02EE0200604F00F0000EB800026
:103AE00005EB800009D5808C20B304F07F0000EB4B
:103AF000800005EB800614360AE0B0F86401C8B116
:103B000004F07F0000EB800005EB800606F5AA7646
:103B10004CB1802C07D021462846FFF73DFD10B15F
:103B20000120306000E03760022231462846FFF76E
:103B3000D0FA02E02846FFF7A7FA4046BDE8F08138
:103B400070B50546087800240E4610F0600003D0DA
:103B5000202801D0402827D195F89C02012803D0C5
:103B6000022801D003281FD1B088C1B201291AD878
:103B7000C1B22846FFF776FAFF280CD058B9D5F81D
:103B8000B8128A683AB1C5F8D4028A683146284624
:103B90009047044600E00324F088204307D12846DC
:103BA000FFF7A4FA03E031462846FFF76DFA2046F6
:103BB00070BD704700487047D416002070B50A7871
:103BC000012302F00F054E78AB401B4CD0F81C5877
:103BD000012E17D045EA0343C0F81C3800EB421011
:103BE000D0F8002B12040BD4D0F8002B8B89097964
:103BF000C3F30A031A4344EA81410A43C0F8002B85
:103C0000002070BD9BB21D43C0F81C5800EB421051
:103C1000D0F800391B04F3D4D0F800398D89097924
:103C2000C5F30A0589042B4341EA82510B43234320
:103C3000C0F80039E4E7000000800010D0F8001957
:103C40006FF30A01C0F80019D0F8041841F480712C
:103C5000C0F804180020704770B5044606990A9E03
:103C6000049D0D98012916D0E06840F04000E06006
:103C7000204600F02BF8A16B1EB321F48031A16324
:103C8000012D07D1A16841F00601A160A16841F0B2
:103C90002001A16070BDA16B21F48031A163E168B6
:103CA000094A1140E160E16821F44011E160012816
:103CB00003D1E06840F48010E060204600F006F890
:103CC000DEE741F48031DAE7BFFFBDFF08B500222F
:103CD0000D490092009B5B1C00938B420CD803693A
:103CE000002BF7DA0092026942F001020261009AA9
:103CF000521C00928A4201D9032008BD0269D207F2
:103D0000F5D1002008BD0000400D030030B54C780F
:103D10000A78012300EB4212012C2CD0D2F8004B80
:103D2000002C0BDAD2F8004B44F00064C2F8004BD0
:103D3000D2F8004B44F08044C2F8004BD0F83C5815
:103D40000C7804F00F0403FA04F425EA0444C0F8E4
:103D50003C48D0F81C48097801F00F018B4024EA58
:103D60000341C0F81C18D2F8000B19490840C2F8EA
:103D7000000B002030BDD2F80049002C0BDAD2F83D
:103D8000004944F00064C2F80049D2F8004944F008
:103D90008044C2F80049D0F83C480D7805F00F0582
:103DA00003FA05F5ADB2AC43C0F83C48D0F81C4866
:103DB000097801F00F018B4099B28C43C0F81C4880
:103DC000D2F8000903490840C2F80009D1E7000011
:103DD0000078F3EF007833ECD0F8001E21F00301F7
:103DE000C0F8001ED0F8041821F00201C0F8041831
:103DF00000207047D0F8001E21F00301C0F8001E1B
:103E0000D0F8041841F00201C0F8041800207047EF
:103E10002DE9F04F00250E460446DDF82CC0DDF8F4
:103E200024B0109F2846294604EB8002C2F80411F2
:103E3000401C0F28F8D32046C7B1806B20F4001235
:103E4000A263A06B40F40022A26308468846C4F82F
:103E5000000ED4F800182046C4F80018BCF1010F79
:103E600016D0D0F8001841F0030116E0D0F804088D
:103E700040F00202C4F80428A06B40F40012A263D0
:103E8000A06B20F40022A263A06B20F48022DBE769
:103E9000D0F800180BB141F00101C0F80018102152
:103EA00000F0EEFA00B10125204600F0CBFA00B197
:103EB00001254046C4F81088C4F81488C4F81C884A
:103EC00000214FF000694FF0904A4FF67F3314E025
:103ED00004EB4112D2F800C9BCF1000F06DA11B1AF
:103EE000C2F800A904E0C4F8009901E0C2F8000992
:103EF000C2F81009C2F80839491C8E42E8D80021DE
:103F000015E000BF04EB4112D2F800CBBCF1000F6A
:103F100006DA11B1C2F800AB04E0C4F8009B01E07E
:103F2000C2F8000BC2F8100BC2F8083B491C8E42C5
:103F3000E8D8D4F8101821F48072C4F81028A061D1
:103F40006FF080406061BBF1000F03D1A06940F0C9
:103F50001000A061A06909490843A0610C9818B13C
:103F6000A06940F00800A061012F03D1A0690449B5
:103F70000843A0612846BDE8F08F000000383C806F
:103F800004000040816821F0010181600020704739
:103F900070B50D784E78444CEBB200EB4313012E14
:103FA00021D0D3F8100B6FF31200C3F8100BD3F825
:103FB000100B2040C3F8100B886908B1C8688861ED
:103FC000C868C861D3F8100B40F40020C3F8100B88
:103FD000D3F8100BCC69C4F312042043C3F8100BC0
:103FE000012A55D058E08E69002ED3F8106932D0DE
:103FF0006FF31206C3F81069D3F810692640C3F8AE
:1040000010698E69CC68A64200D98C61D3F810493A
:1040100044F40024C3F81049D3F810498E69C6F35C
:1040200012063443C3F81049012A22D000EB45128E
:10403000D2F8003943F00443C2F800398A6932B338
:10404000D0F83428097801F00F03012199400A4380
:10405000C0F8342826E02640C3F81069D3F8104988
:1040600044F40024C3F81049D3F810496FF3120444
:10407000D8E7496919B100EB4512C2F8141900EBF1
:104080004510D0F8001941F00441C0F8001909E0CA
:10409000086908B1C3F8140BD3F8000B40F00440D2
:1040A000C3F8000B002070BDFFFF07E010B5036CE4
:1040B000134CA34203D9D0F8003B002B1EDB002396
:1040C000C0F8103BD0F8103B43F40023C0F8103B7D
:1040D000D0F8103B43F01803C0F8103BD0F8103B69
:1040E00043F0C043C0F8103B012907D1C0F8142B9E
:1040F000D0F8001B41F08021C0F8001B002010BD4B
:104100000A30544F4A780B78012A00EB43100BD049
:10411000D0F8002B22F40012C0F8002B09790329F3
:1041200014D0022912D017E0D0F8002922F400128E
:10413000C0F800290979032901D002290CD1D0F84F
:10414000001941F08051C0F8001905E0D0F8001BBB
:1041500041F08051C0F8001B002070470A784B786E
:10416000D1B200EB4110012B12D0D0F8001B002976
:1041700006DB2AB1D0F8001B21F08041C0F8001BFB
:10418000D0F8001B41F40011C0F8001B002070475C
:10419000D0F80019002906DB2AB1D0F8001921F067
:1041A0008041C0F80019D0F8001941F40011C0F89E
:1041B0000019EBE7F8B50C784F78764DE3B26FF065
:1041C000604600EB4313012F27D0D3F8104B6FF359
:1041D0001204C3F8104BD3F8104B2C40C3F8104B0B
:1041E0008D69002D75D0CC6825446D1EB5FBF4F5A6
:1041F000ADB26C43CC61D3F8104B06EAC5452C43F5
:10420000C3F8104BD3F8104BCD69C5F312052C43FE
:10421000C3F8104B012A71D0A4E08F691FB3D3F803
:1042200010796FF31207C3F81079D3F810792F4083
:10423000C3F810798F69CD682F447F1EB7FBF5F561
:1042400006EAC545D3F810693543C3F81059D3F8C9
:1042500010598E69C6F312063543C3F810590D790B
:10426000012D10D01BE0D3F810692E40C3F810695F
:10427000D3F8105945F40025C3F81059D3F8105954
:104280006FF3120509E0D3F8105925F0C045C3F8C3
:104290001059D3F8105945F00055C3F81059012AA8
:1042A00018D000EB4413D3F8004944F00444C3F899
:1042B00000490C79012C2FD08A6962B3D0F83428D8
:1042C000097801F00F03012199400A43C0F834280E
:1042D0005EE036E04A691AB100EB4413C3F81429D2
:1042E000097901290FD1D0F80818C90500EB44114C
:1042F000D1F8002903D442F0005202E02EE042F04F
:104300008052C1F8002900EB4410D0F8001941F0A8
:104310000441C0F800193BE0D0F80848E405D3F8A0
:10432000004902D444F0005401E044F08054C3F842
:10433000004900920A8B93B20A78096900F0D0F91B
:1043400026E0D3F8104BCD68C5F312052C43C3F813
:10435000104BD3F8104B44F4002459E70A690AB112
:10436000C3F8142B097901290CD1D0F80808C0052D
:10437000D3F8000B02D440F0005001E040F0805030
:10438000C3F8000BD3F8000B40F00440C3F8000B57
:104390000020F8BDFFFF07E038B500220092134669
:1043A0004D780A7842F2107400EB4212012D19D0B8
:1043B000D2F8005B002D3CDAD2F8005B45F00065D6
:1043C000C2F8005B0A7800EB4212D2F8005B45F0BD
:1043D0008045C2F8005B009A521C0092A24221D98B
:1043E000012326E0D2F80059002D22DAD2F8005934
:1043F00045F00065C2F800590A7800EB4212D2F885
:10440000005945F08045C2F80059009A521C0092AC
:10441000A242E5D80A7800EB4212D2F80029002A1D
:10442000F3DB06E00A7800EB4212D2F8002B002AF8
:10443000D1DB184638BD816841F001018160002060
:104440007047000008B500220C490092009B5B1CDD
:1044500000938B420AD80369002BF7DA00921022EE
:104460000261009A521C00928A4201D9032008BDC1
:104470000269D206F5D4002008BD0000400D0300FB
:1044800018B500230D4A0093009C641C00949442CC
:104490000CD80469002CF7DA0093202343EA811139
:1044A00001610099491C0091914201D9032018BD76
:1044B00001698906F5D4002018BD0000400D0300F5
:1044C000D0F8080810F0060004D0022803D006280F
:1044D00001D00F20704702207047406900F00100B2
:1044E0007047D0F81818D0F81C08084080B2704700
:1044F000D0F81818D0F81C080840000C704710B508
:10450000D0F81038D0F8342801F00F0400EB411037
:10451000E24002F00102D0F8080943EAC21210405A
:1045200010BD00EB4111D1F8081BD0F81408084069
:104530007047416980690840704730B503460846B6
:10454000940802F00301002203F5805303E01D6884
:1045500040F8045B521CA242F9D300290BD01C681E
:104560000022D50024FA05F3491E521C090400F864
:10457000013B090CF5D130BD70B50446C06800257B
:1045800020F0C040E060012901D079B120E0E0686E
:1045900040F00050E0600120FCF75CFA60696D1C9F
:1045A00010F0010F10D1322DF5D30DE0E06840F08E
:1045B0008040E0600120FCF74DFA60696D1C10F04E
:1045C000010F01D0322DF5D3322D01D0002070BD66
:1045D000012070BDD0F8002822F4FE62C0F8002847
:1045E000D0F800284FF4FE6303EA01110A43C0F833
:1045F0000028002070470000022A3ED1264A274B9F
:104600000A449A4201D20F2138E0254A254B0A4438
:104610009A4201D20E2131E0234A244B0A449A42A5
:1046200001D20D212AE0224A224B0A449A4201D2A9
:104630000C2123E0204A214B0A449A4201D20B214B
:104640001CE01F4A1F4B0A449A4201D20A2115E07E
:104650001D4A1E4B0A449A420FD31D4A1D4B0A4461
:104660009A4201D2082109E01B4A11441B4A914297
:1046700001D2072102E0062100E00921C26822F4EC
:104680007052C260C2684FF4705303EA81210A433A
:10469000C260002070470000405327FF00350C0027
:1046A000401E1BFF40420F0000DC0BFF804F12003A
:1046B000808CF9FE20D6130060B6E5FE60E316009C
:1046C00000D3CEFE40771B00C05BB3FEC09121003B
:1046D00000CA91FE20753800E05459FEE09C41006C
:1046E00010B5029C74B9DB1C9C0800EB023000235F
:1046F00000F5805004E000BF51F8042B02605B1C01
:10470000A342F9D3002010BDFEE70907090E0028D7
:1047100004DB00F1E02080F80014704700F00F0087
:1047200000F1E02080F8141D7047704770B54FF01D
:10473000E024002265690949A36909684843A16921
:104740009942FCD002D2A3EB010302E0A5EB0106E3
:1047500033441A440B468242F1D370BD100100204D
:10476000FCF7B2FAFEF778F8FDF75CFE4FF47A70CA
:10477000FCF770F9FDF746FF1E20FCF76BF9FDF71B
:10478000D7FEFDF707FFFDF721FFFBF719FF0848EC
:10479000FDF7E0FBFCF7C8F8064C0025207801285F
:1047A000FCD1FDF7EDFDFEF71DF82570F6E70000E2
:1047B000280100201F0100204FF04070E1EE100A98
:1047C000704700000000000000000102030406071B
:1047D000080900000000010203040000FC47000873
:1047E0000000002028010000C4010008244900083E
:1047F0002801002078650000E0010008B1320008BF
:10480000E1320008ED32000815330008413300089A
:1048100091320008BD3200080403090412010002AD
:10482000020200408304405700020102030100001D
:104830001A0300000000000000000000000000005B
:10484000000000000000000000000000A1080008B7
:104850009D0800085B080008C5080008F908000862
:104860000100000010000000000000000024F4001F
:1048700000000000810182000A06000200000040E2
:104880000100000009024300020100C032090400D7
:1048900000010202010005240010010524010001AD
:1048A0000424020205240600010705820308001003
:1048B00009040100020A000000070501024000008F
:1048C0000705810240000000892D0008FD2B00082B
:1048D000272F0008000000008D2C0008492B00083D
:1048E000BF2B0008000000000000000000000000D6
:1048F0000D2D0008D12C00084D2D0008C52C0008F6
:10490000000004000000000004000000000000009F
:10491000030200030000000000000000000000008F
:044920000000000093
:040000050800018965
:00000001FF
